:020000040800F2
:10000000C806002091010008AD0A0008A90A0008EE
:10001000AB0A000807070008C5150008000000002B
:100020000000000000000000000000006D0E00084D
:10003000B508000800000000510B0008710E000810
:10004000AB010008AB010008AB010008AB010008E0
:10005000AB010008AB010008B9080008AB010008BB
:10006000AB010008AB010008AB010008AB010008C0
:10007000AB010008AB010008AB010008AB010008B0
:10008000AB010008AB010008AB010008AB010008A0
:10009000AB010008AB010008AB010008AB01000890
:1000A000AB010008AB010008AB010008AB01000880
:1000B000AB010008AB010008590F0008AB010008B4
:1000C000AB010008AB010008AB010008AB01000860
:1000D000AB01000819140008AB010008AB010008CF
:1000E000AB010008AB010008AB01000800F002F80A
:1000F00000F03EF80AA090E8000C82448344AAF184
:100100000107DA4501D100F033F8AFF2090EBAE881
:100110000F0013F0010F18BFFB1A43F0010318473B
:10012000701E0000901E0000103A24BF78C878C1ED
:10013000FAD8520724BF30C830C144BF04680C60ED
:10014000704700000023002400250026103A28BF35
:1001500078C1FBD8520728BF30C148BF0B60704739
:100160001FB59DE8030000F007F91FBD10B510BDD5
:1001700000F0C0F81146FFF7F3FF01F092FE00F027
:1001800031F903B4FFF7F2FF03BC01F087FE000072
:100190000948804709480047FEE7FEE7FEE7FEE71B
:1001A000FEE7FEE7FEE7FEE7FEE7FEE70448054957
:1001B000054A064B70470000890E0008ED00000854
:1001C000C8000020C8060020C8020020C802002085
:1001D0007047002000F008F8FFF7C8FF012001F089
:1001E0005DFE70477047704710B500F065F8BDE8D8
:1001F000104000F05BB800000048704798000020F5
:1002000070B5064600F09CF8056806F10B0020F07A
:100210000704B4429CBF002070BD2B466A68BAB187
:100220001068A04210D304F1080188423CBF506816
:10023000586007D35168101941601168091B0160AB
:1002400058601460101D70BD13465268002AE7D133
:100250002146284600F07CF80028DED170BD70B53C
:100260000446051F00F06CF80068002C14BF4468B9
:1002700070BD002C18BFAC423CBF20466468F8D368
:1002800001680A18AA4218BF456003D12A680546CA
:100290001144016028684119A1421CBF6C6070BD07
:1002A0006168696021680844286070BD002801D039
:1002B00001F0F4BD7047000010B5002102A000F06D
:1002C00097F8012010BD0000534947414252543A6B
:1002D0002041626E6F726D616C207465726D696E23
:1002E0006174696F6E00000000F09BB800487047B1
:1002F000640000207546FFF7F9FFAE460500694629
:10030000534620F00700854618B020B5FFF74EFF92
:10031000BDE820404FF000064FF000074FF0000806
:100320004FF0000B21F00701AC46ACE8C009ACE887
:10033000C009ACE8C009ACE8C0098D4670470000B0
:10034000004870476C000020704770477047704746
:1003500038B504460A4600206946AFF300800028FD
:1003600008BF38BD02460099204600F067F801201A
:1003700038BD012000F07CB8F8B5AFF30080054629
:1003800000200C46102000BF0646A819A0420DD937
:10039000324669460020AFF30080070008BF00F036
:1003A00067F80098A04218BF0546C419FFF7C8FFB8
:1003B00005600746F01D20F007004619284600F0AA
:1003C0000AF8B44208BFF8BDA21B31463868BDE840
:1003D000F84000F033B800210160C0E90110704717
:1003E000102070470446AFF300802046FFF7C9FE97
:1003F00070B505460C460A2000E06D1C01F04FFD6B
:1004000035B128780028F8D102E0641C01F047FDDE
:1004100014B120780028F8D1BDE870400A2001F01E
:100420003EBD10B500F02FF8016919B1002202613C
:10043000884701E080688047FFF7CBFE03464068AD
:100440008C46002818BF88423CBF03464068F8D35A
:1004500018681844884207D00CF1030020F0070008
:10046000001D411A521A0146081D0A60FFF7F7BE27
:1004700010B500F031F8BDE81040FFF717BF0000DD
:1004800010B5FFF7A6FE70B500F022F80468054627
:10049000A4B92020FFF7B4FE040011D009490020C0
:1004A0002C60C4E900010849A160207320616061EB
:1004B0000649A06109B100F037F8E061204670BD3F
:1004C000FFF787FE00000000810400080000000024
:1004D00000487047A000002010B5012805D0002179
:1004E00003A0FFF785FF012010BD09A1F8E7000078
:1004F00053494752544D454D3A204F7574206F660D
:100500002068656170206D656D6F72790000000074
:100510003A2048656170206D656D6F727920636F58
:10052000727275707465640010B58820FFF768FEFC
:10053000002801D00021017010BD802902D808B127
:10054000017809B100207047012100F8081B7047AD
:1005500018B100F10802914201D00020704700213B
:10056000017070470029816814BF41F0010121F03A
:1005700001018160704710B5A0F18041B1F5923161
:1005800011D0B1F5806119D0B1F5A05118BF10BDDF
:100590000121C80300F018FBBDE8104000214FF412
:1005A000004000F011BB0121480200F00DFBBDE846
:1005B000104000214FF4007000F006BB01218802BA
:1005C00000F002FBBDE8104000214FF4806000F015
:1005D000FBBA0029816814BF41F4801121F4801115
:1005E0008160704701460020896811F0040F18BF30
:1005F00001207047C06C80B270470246002012682C
:100600000A4218BF0120704701460020896811F096
:10061000080F18BF012070474268D1E9003C22F45E
:10062000807222F4702242EA0C221A4342608268ED
:100630000A4B1A40D1E903C343EA0C03D1F808C0BE
:1006400042EA4C021A438260C26A097D22F47002B7
:10065000491EC9B242EA0151C1627047FDF7F1FF7C
:1006600030B4072409290DD9C568A1F10A0C0CEB97
:100670004C0C04FA0CF425EA040403FA0CF32343AB
:10068000C3600AE0056901EB410C04FA0CF425EAA9
:10069000040403FA0CF3234303611F23072A0CD23B
:1006A000D0F834C0521E02EB820293402CEA0303BE
:1006B00091401943416330BC70470D2A0CD2D0F8E9
:1006C00030C0D21F02EB820293402CEA0303914018
:1006D0001943016330BC7047D0F82CC00D3A02EBCF
:1006E000820293402CEA030391401943C16230BC5B
:1006F0007047816841F0080181607047816841F06E
:10070000040181607047FEE7054A012303FA00F007
:100710000029116814BF084321EA000010607047E7
:100720000074004010B50121480700F035FABDE81B
:10073000104000214FF0005000F02EBA0B4B10B4C7
:100740001A6840F6FE7C0CFA00FC22EA0C02D1E9A1
:1007500000C44CEA040CD1E9024121434CEA0101F6
:1007600001FA00F01043186010BC7047007400409C
:10077000A0F6F83081B000F1804000F50040009014
:10078000016001B07047A0F6EC3081B000F180400C
:1007900000F500400090016001B07047044A002954
:1007A000516814BF084321EA000050607047000000
:1007B000002004E0016821F00101016000210160D6
:1007C00041608160C1602E4A2E49904204BF486852
:1007D00040F00F0022D02C4A904204BF486840F0FD
:1007E000F0001BD0294A904204BF486840F4706072
:1007F00014D0274A904204BF486840F470400DD09E
:10080000244A904204BF486840F4702006D0224A2F
:10081000904204BF486840F4700001D148607047BE
:100820001E4A904204D1486840F0706048607047AA
:100830001B4A111F904204BF086840F00F0014D0FB
:10084000184A904204BF086840F0F0000DD0164AE4
:10085000904204BF086840F4706006D0134A90428A
:1008600004BF086840F4704001D108607047104A26
:10087000904218BF7047086840F4702008607047C5
:1008800008000240000002401C000240300002400C
:1008900044000240580002406C00024080000240C8
:1008A000080402401C040240300402404404024098
:1008B000580402407047000002490120087000F00F
:1008C00003B80000200000200149086070470000C4
:1008D00014040140C2680168002A35D01F4A136819
:1008E00023EA01011160111D0A6803689A430A6036
:1008F000416801F1804101F582310A6803681A43B9
:100900000A6017490A6803689A430A600B1D1A684F
:10091000D0F800C022EA0C021A608268102A08D0BF
:1009200002F1804202F582321168006808431060CB
:1009300070470A68D0F800C042EA0C020A601968E1
:100940000068084318607047406800F1804000F577
:100950008230026822EA0101016070470004014010
:10096000080401408A0721F0030101F1804101F5EB
:100970008031120F0F23D1F808C093402CEA0303F3
:100980008B608B6890401843886070472DE9F001B8
:100990000B7A002203F00F0C13F0100F1CBF4B68F2
:1009A00043EA0C0C0B784FF00F0613F0FF0F4FF0DB
:1009B000010518BF046819D00F8805FA02F31F401B
:1009C0009F420FD1970006FA07F824EA08040CFAB0
:1009D00007F73C438F68282F08BF436102D0482F98
:1009E00008BF0361521C082AE6D304600A88FF2A64
:1009F00087BF44680022BDE8F001704702F1080398
:100A00000F8805FA03F31F409F420FD1970006FAA3
:100A100007F824EA08040CFA07F73C438F68282FEC
:100A200008BF43618F68482F08BF0361521C082A22
:100A3000E4D34460BDE8F0017047000070B4194A87
:100A400010F0004F14BFD3695368C0F303444FF450
:100A5000401C3CEA00054FEA505C4FEA0C1C86B291
:100A600006FA0CFC16D010F4801F08BF23EA0C0312
:100A700003D0032505FA04F4A34343F0706300296F
:100A800018BF4CEA030310F0004F14BFD36153604A
:100A900070BC7047546823F0706324F07064546035
:100AA000EDE7000000000140FEE7FEE7FEE7000082
:100AB00010B401784268012322B3184A12680F2447
:100AC00002F4E062C2F5E062120AC2F1040C24FAF8
:100AD00002F2447801F1E02104FA0CFC847822400F
:100AE00042EA0C02120181F80024007800F01F0194
:100AF00003FA01F14009800000F1E020C0F8001184
:100B000010BC704701F01F0003FA00F0490989008A
:100B100001F1E021C1F8800110BC70470CED00E04C
:100B2000094A136823F0030318431060074802685A
:100B300042F00402026001290CBF30BF20BF0168EF
:100B400021F00401016070470070004010ED00E0EA
:100B50007047000003494A6822F44042104348604D
:100B60007047000000100240044A0029516914BF78
:100B7000084321EA00005061704700000010024065
:100B8000044A0029D16914BF084321EA0000D0615A
:100B90007047000000100240044A0029116914BF88
:100BA000084321EA00001061704700000010024075
:100BB000044A0029916914BF084321EA00009061AA
:100BC0007047000000100240044A0029D16814BF99
:100BD000084321EA0000D060704700000010024086
:100BE000264910B44A6812F00C03254A18BF042B9A
:100BF00019D0082B17D14B68D1F804C003F4701337
:100C00004FF002041CF4803F04EB934304BF1D4AE1
:100C10005A4308D0D1F82CC00CF00F0C0CF1010C89
:100C2000B2FBFCF25A4302604A680F2303EA121235
:100C3000154B9A5CD0F800C02CFA02F24260D1F851
:100C400004C0072404EA1C2C13F80CC022FA0CFC84
:100C5000C0F808C0D1F804C004EADC2C13F80C304A
:100C6000DA40C2604968032303EA9131074B595CBB
:100C7000B2FBF1F1016110BC7047000000100240AE
:100C800000127A0000093D0004000020000000204E
:100C9000002243090949012B08BF096803D0022B30
:100CA0000CBF096A496A00F01F00012303FA00F033
:100CB000084218BF01221046704700000010024091
:100CC0000248406800F00C0070470000001002402D
:100CD0000C490A6822F480320A600A6822F48022F1
:100CE0000A60B0F5803F04BF086840F4803006D049
:100CF000B0F5802F06BF086840F4A0207047086058
:100D0000704700000010024001490866704700006B
:100D10000000424203494A6822F00302104348603F
:100D2000704700000010024081B000200B49009085
:100D300000200A6812F4003F18BF0120009A521CDC
:100D40000092B2F5A06F01D00028F1D0086810F42D
:100D5000003018BF012001B07047000000100240B1
:100D600010B504460B4884B0012150F82400FFF769
:100D70001FFF0948694630F81400ADF80000102044
:100D8000029003200190054850F82400FFF7FEFD73
:100D900004B010BD4C1F0008421F000818000020BE
:100DA0000349044A31F8101052F82000416170479D
:100DB000421F0008180000200349044A31F81010AF
:100DC00052F8200001617047421F000818000020FF
:100DD00030B504461F480D4689B050F82400012163
:100DE00040F00100FFF7E4FE042008901A4806A92D
:100DF00030F81400ADF81800184850F82400FFF738
:100E0000C5FD012D1CBF09B030BD154810F81410E8
:100E1000801C10F81400FFF7A5FD1248012530F8DA
:100E200014000090002001900820CDE902056846DA
:100E3000FFF750FD0C4810F814008DF810000F203B
:100E40008DF811008DF8120004A80595FFF730FE0B
:100E500009B030BD481F00083C1F000814000020E6
:100E6000381F00083E1F0008401F000870470000A0
:100E70000448807800284FF0000001D0FFF79CBFA5
:100E8000FFF78EBF20000020304882B0016841F09B
:100E90000101016041682E4A11404160016821F45E
:100EA000102121F080710160016821F4802101602E
:100EB000416821F4FE0141604FF41F01816000226E
:100EC000C26201920092016841F4803101600168C0
:100ED00001F4003100910199491C0191009919B95F
:100EE0000199B1F5A06FF2D1016811F4003F08BF7C
:100EF000009224D001210091416841604168416025
:100F000041684160416821F47C114160416841F4CD
:100F100098114160016841F080710160016811F031
:100F2000007FFBD0416821F003014160416841F03E
:100F300002014160416801F00C010829FAD105491C
:100F40004FF00060086002B07047000000100240DF
:100F50000000FFF808ED00E010B50A4C0221204621
:100F600000F025F9002808BF10BD0221204600F03E
:100F700016F80549012048702046BDE810400021C0
:100F800000F010B80008004020000020002901886F
:100F900014BF41F0800121F0800101807047C943F6
:100FA000018270470029018814BF41F0010121F03E
:100FB0000101018070470029B0F8441014BF41F4CA
:100FC0000041C1F30E01A0F84410704710B5A0F124
:100FD0008041B1F596313BD0B0F1804F4DD011F545
:100FE000943140D0B1F5806151D0B1F5806158D0D5
:100FF000B1F580615FD0B1F5806166D0B1F5903117
:101000006DD0B1F5C05175D0B1F580617DD0B1F52D
:1010100080617DD011F59E317BD0B1F5806179D0B2
:10102000B1F5806177D0B1F5903175D0B1F58061BF
:1010300073D0B1F5806118BF10BD01218804FFF79E
:10104000C3FDBDE8104000214FF48020FFF7BCBD78
:101050000121C802FFF7B8FDBDE8104000214FF4A0
:101060000060FFF7B1BD01210220FFF795FD0021CF
:10107000BDE810400220FFF78FBD01210846FFF7B1
:101080008BFD0021BDE810400120FFF785BD012147
:101090000420FFF781FD0021BDE810400420FFF788
:1010A0007BBD01210820FFF777FD0021BDE810403E
:1010B0000820FFF771BD01211020FFF76DFD002111
:1010C000BDE810401020FFF767BD01212020FFF789
:1010D00063FD0021BDE810402020FFF75DBD012128
:1010E0004803FFF771FDBDE8104000214FF40050A8
:1010F000FFF76ABD0121C804FFF766FDBDE8104097
:1011000000214FF40020FFF75FBD0121080505E035
:101110000DE017E020E029E033E03DE0FFF754FD6B
:10112000BDE8104000214FF48010FFF74DBD0121B4
:101130004805FFF749FDBDE8104000214FF40010BD
:10114000FFF742BD01214020FFF726FD0021BDE849
:1011500010404020FFF720BD01218020FFF71CFD3B
:101160000021BDE810408020FFF716BD01210802D4
:10117000FFF712FDBDE8104000214FF48070FFF72B
:101180000BBD01210804FFF71FFDBDE81040002141
:101190004FF48030FFF718BD01214804FFF714FD1C
:1011A000BDE8104000214FF40030FFF70DBD038A69
:1011B000002280890B4200EA01001CBF00280122A6
:1011C00010467047002A828914BF114322EA0101A8
:1011D0008181704710B4028C22F001020284028CDB
:1011E0008388B0F818C00C882CF0730C44EA0C0CFF
:1011F0000C8922F0020222434C882243A0F1804451
:10120000B4F596341CBFA0F18044B4F59A340DD0E7
:10121000A0F18044B4F5A0341FBFA0F18044B4F520
:10122000A234A0F18044B4F5A4340DD14C8922F04D
:10123000080222438C8822F0040222438C8923F482
:1012400040732343CC8923438380A0F818C0C98806
:101250008186028410BC704730B4028C22F01002E8
:101260000284038CB0F804C0028B0D8822F4E6449B
:101270004FF6FF7202EA05252C430D8923F0200367
:1012800002EA05152B434D8802EA05152B43A0F110
:101290008045B5F596351CBFA0F18045B5F59A356A
:1012A00017D14D8923F0800302EA05152B438D8861
:1012B00023F0400302EA05152B438D892CF4406C82
:1012C00002EA850545EA0C0CCD8902EA850242EA6C
:1012D0000C0CA0F804C00483C9880187038430BCC7
:1012E000704730B4028C22F480520284048C8288CD
:1012F000838B0D8823F4E64C4FF6FF7303EA052534
:1013000045EA0C0C0D8924F4005403EA05352C43FE
:101310004D8803EA05352C43A0F18045B5F5963597
:101320001CBFA0F18045B5F59A3505D18D8922F411
:10133000804203EA85131A438280A0F81CC0C98842
:10134000A0F84010048430BC7047828B4FF6FF73C6
:1013500022F4006203EA01211143818370478185F1
:101360007047A0F84010704710B40288234BDFF894
:1013700090C0984218BF604511D0B0F1804F1CBF9B
:10138000A0F18044B4F5806409D0A0F18044B4F5A4
:1013900000641CBFA0F18044B4F5406403D14C88C4
:1013A00022F070022243A0F18044B4F580541CBFA7
:1013B000A0F18044B4F5A05403D0CC8822F440724C
:1013C000224302808A8882850A880285984218BF53
:1013D00060450DD0A0F18042B2F5A0321FBFA0F150
:1013E0008042B2F5A232A0F18042B2F5A43201D11E
:1013F000097A01860121818210BC7047002C0140CE
:10140000003401404FF6FF71818000210180C180CE
:1014100041800172704700000F48018811F0200FD1
:1014200008BF704710B5018821F0200101800B49E9
:1014300009880B4CCAB261680A4B0B44491C6160B5
:101440001A70712A18BF10BD00216160322100F0AE
:10145000B2F80120207010BD00380140043801406E
:101460002400002058000020028A4FF2FF031A4097
:101470000B88B1F802C043EA0C03B1F804C0C98874
:101480004CEA010119431143018270470021018098
:1014900041808180C18070470029818914BF41F457
:1014A000005121F4005181817047002A828A14BFC3
:1014B000114322EA010181827047C1F3421301F016
:1014C0001F014FF0010C0CFA01F1012B08BF0C3089
:1014D00003D0022B0CBF10301430002A026814BF56
:1014E000114322EA010101607047000030B5044653
:1014F000008A85B00D464CF6FF710840E988084324
:101500002082A0894EF6F3110840A9882A89114348
:101510006A8910430843A081A08A4FF6FF41084022
:10152000A9890843A0826846FFF75AFBA4F18040CE
:10153000B0F59C300CBF03980298A18911F4004FBC
:1015400000EBC00101EB0010296814BF49008900BD
:10155000B0FBF1F0114A6FF0180CA2FB0031490901
:1015600009010B0903FB0CF300EB8300A38913F4BF
:10157000004F4FF0320314BF03EBC00003EB001029
:10158000A2FB00204FEA501014BF00F0070000F04B
:101590000F000843208105B030BD00001F85EB51CE
:1015A0004FF41651016000218180C18001810C221D
:1015B000428181817047C9B28180018811F0800F1A
:1015C000FBD07047FEE700002DE9F05F827D012A25
:1015D0007ED1C269931CC0E906231180B0F814C003
:1015E0000169C36901EB4C029A4208BFC16184885A
:1015F000076A002C6CD08669056800F1100836F97E
:101600000229B5F900906FF0010386618E4204D281
:1016100003EB4C060E44C8F8086009FB02F9012CE4
:1016200056D98669B5F9028000F1100A36F9022907
:101630008661B14204D903EB4C060E44CAF8086037
:1016400008FB029A022C43D98669B5F9048000F19F
:10165000100936F902298661B14204D903EB4C0620
:101660000E44C9F8086008FB02A9032C78D98669E2
:10167000B5F9068000F1100A36F902298661B142F7
:1016800004D903EB4C060E44CAF8086008FB029626
:1016900004224FF00109B846012F88BFC64653D92E
:1016A00094425DD9D0F8188035F912B000F1100AD3
:1016B00038F90279C0F81880414504D903EB4C0889
:1016C0008844CAF808800BFB076B561CB44200E044
:1016D00046E045D9876935F916A000F1100837F9B9
:1016E00002698761B94204D903EB4C070F44C8F87B
:1016F00008700AFB06BB961CB44231D935F916A016
:1017000037F90269C8F80870B94204D903EB4C07ED
:101710000F44C8F808700AFB06BAD61CB4421FD999
:1017200035F916B037F90269C8F80870B94204D91A
:1017300003EB4C070F44C8F808700BFB06A6121DFC
:1017400009F10109F145ABD3D0F824B04FF00008FE
:10175000BBF1000F1DD900BF08EB0207BC4201D846
:10176000FEF737FDD0F818E035F917A000F11009A1
:101770003EF90279C0F818E0714504D903EB4C0E2C
:101780008E44C9F808E00AFB076608F10108C34562
:10179000E2D846F3CF30BDE8F09F00002DE9F041DC
:1017A0000E460904090C026081804FF00005857126
:1017B0008260C26035D000F11004701C87B27800DE
:1017C00000F054FB2060A7800120A0712068A06079
:1017D000E06037B3A088AA1E216802EB40020A44E9
:1017E000B0F1004F1FD20128D8BF012001DD002831
:1017F0000EDD921C10F0010F18BF22F8025D4010A0
:1018000006D000BF22F8025C22F8045D401EF9D128
:10181000B108216106F00301A4F110006161BDE887
:10182000F081FEF7D6FC22F80259401EFBD1EFE70B
:101830000446032100F058F8012104F5827000F0FD
:101840009BF900BF04F5827000F0EAFA01B204F5DA
:101850008870FFF7B9FE00F5006081B204F5807072
:1018600000F0EEFAEEE7000010B5042100F060F899
:10187000064A1F2100F58870FFF790FFA0F58874D5
:1018800064210C3800F046F9204610BDF81E00080F
:1018900010B50446134A00200029107004BF30BF61
:1018A00010BD02210120FFF73BF94FF48030FFF714
:1018B0000FFAFFF739FAC4F80C01012818BF10BD60
:1018C0000120FFF721FA3920FFF7E2F90028FAD0CA
:1018D0000220FFF71FFA00BFFFF7F2F90828FBD13B
:1018E00010BD00002000002070B5052901DBFEF7C7
:1018F00070FC0D4899B10D4A054632F8114001219E
:10190000FFF750FB4FF6FF7000EA44012846FFF74F
:1019100026FD21462846BDE87040FFF722BDBDE800
:1019200070400021FFF73EBB00040040541F000838
:101930002DE9F0430C468BB0014600F003FA00227B
:10194000214600F5807000F0C7F905222146001DF0
:1019500000F016F9A0F5827672B660490868604A10
:10196000012520F00100136843F0807313605E4B83
:101970005C4A1A6008605D4B00241C605C4A0227C8
:1019800042F8F07F4FF0070C42F8E0CCDFF864C17A
:10199000CCF80040DFF86481DFF85CC1C8F800C013
:1019A0004FF4807CC2F814C2554A1A6040F001001E
:1019B00008600020FFF7D4F90020FFF7F1F90120BB
:1019C000FFF7CEF90120FFF7EBF901210020FFF727
:1019D000FFF901210846FEF7E1FE01210220FEF792
:1019E000DDFE0121C802FEF7D9FE01210420FFF728
:1019F000C7F8DFF810914846FFF7E8FA4FF6FF7096
:101A0000ADF8040042F6E068ADF80080ADF806409D
:101A1000ADF8024069464846FFF7A6FC1020ADF835
:101A20001000ADF81250ADF8184004A94846FFF771
:101A3000D1FB1E208DF820008DF8224004208DF867
:101A4000210008A80995FFF733F801220221484632
:101A5000FFF7B8FB01210220FFF792F86802ADF80A
:101A60001C001820CDE9087007A92748FEF78EFF53
:101A700001212648FEF7E2FF254F3846FFF7A6FA78
:101A80004FF47A70ADF81000ADF81480ADF8164040
:101A9000ADF8124004A93846FFF766FC6020ADF8A7
:101AA000000041F27070ADF80600ADF80250ADF8DC
:101AB000084069463846FFF714FC08213846FFF70E
:101AC00044FC01213846FFF761FA01213846FFF74F
:101AD00069FA62B630460BB0BDE8F083000E00E054
:101AE000FCED00E055CEACC5B00F00E0800E00E08C
:101AF000000004E0400E00E0FE030040001000E0A3
:101B00000D0001000008004000100140000C1A0008
:101B10000004004010B504464FF6FF7088B08142C3
:101B200001D3FEF756FBA1806846FFF76BFCA08847
:101B3000ADF804001820ADF800000020ADF8060054
:101B4000ADF8020069462068FFF70EFC6020ADF892
:101B500010000120ADF81200A088ADF81600022098
:101B6000ADF8180004A92068FFF776FB0121206872
:101B7000FFF721FA08B010BD0068FFF713BA0000A4
:101B8000F0B5054691B04FF0804028600C46AA8021
:101B900001214015FFF70CF80020FEF7DBFF4B4F4B
:101BA000002CD7E903017A691092CDE90E0108BF34
:101BB00040200AD0012C08BF022006D0022C03D0FE
:101BC000042C08BF802000D00420ADF838000EA9F6
:101BD0003F48FEF7DBFE002C08BF062407D0012C8F
:101BE00018BF022C03D0042C0CBF07240224394E4A
:101BF0003046FEF7C0FC07F118000FC88DE80F0053
:101C0000D7E90A01CDE9040169463046FEF704FD33
:101C10000723012221463046FEF722FD01213046EE
:101C2000FEF7D7FC01210846FEF7AAFFA8884FF669
:101C3000FF712C46884204D24FF47A725043884296
:101C400001D3FEF7C6FAA08006A8FFF7DBFBA08849
:101C5000ADF81C001820ADF818000020ADF81E00EB
:101C6000ADF81A0006A92068FFF77EFB6020ADF8EA
:101C700028000120ADF82A00A088ADF82E0002202F
:101C8000ADF830000AA92068FFF7E6FA01212068C4
:101C9000FFF791F9012134463046FEF763FC00213D
:101CA0002868FFF77FF92046FEF723FD2046FEF760
:101CB000ABFC0028FAD12046FEF720FD2046FEF7B7
:101CC00091FC0028FAD111B02846F0BD601F000831
:101CD000000801400024014030B587B00C46016087
:101CE000054601214807FEF74BFFFEF71BFD134A8F
:101CF000002CD2E9000192680692CDE904010CBFE4
:101D000020201020ADF8100004A90D48FEF73EFE7B
:101D1000002000900190029003904CB16946FEF7BC
:101D20000DFD00200121FEF7EFFC07B0284630BD75
:101D300010206946FEF702FD1020F3E7601F00083F
:101D4000000801402DE9F04104468CB00830606085
:101D500000260125A4F8F86084F8FA50C4F8FC10B5
:101D600029462846FEF700FF012144F20400FEF751
:101D70001FFF182002904FF49050DFF89880ADF8C4
:101D800000000227694640460197FEF7FFFD482004
:101D900002904FF44060ADF800006946404601975C
:101DA000FEF7F4FD0AA8FFF771FB1B4F0AA938469E
:101DB000FFF75AFB04A8FFF7F3FB4FF461200490F0
:101DC0004FF44070ADF81C0004A93846FFF78EFBB5
:101DD00025208DF820008DF822608DF8215008A86C
:101DE0000995FEF765FE012240F225513846FFF7BE
:101DF00064FB012280213846FFF757FB0748FEF7B6
:101E0000D9FC01213846FFF747FB0CB02046BDE85E
:101E1000F081000000080140003801404400024009
:101E200010B5064C02212046FEF7E7FB0028F9D04A
:101E30002046BDE81040FEF7DDBB00000024014055
:101E4000B1F5805F28BF40F6FF71006800284FF0B1
:101E5000000001D0FEF78CBCFEF795BC10B500F079
:101E600001F810BD10B5FEF7FAF910BD10B500F07D
:101E700001F810BD10B5040007D1012405E0FEF7FC
:101E8000BBF9006800B9044880472046FEF7B8F95E
:101E90000028F4D010BD0000E9020008FEE700F0C1
:101EA00021B800B5CFB06846FFF7DEFC00216846D8
:101EB000FFF71AFD00216846FFF7EAFC6846FFF7C6
:101EC000B7FC9DF82601012804BF4898FFF7C6FF1C
:101ED0009DF81601012804BF4498FFF7BFFF0020BA
:101EE0004FB000BD10B5C4B221460248FFF763FBF6
:101EF000204610BD00380140BFFF3A00A300BEFFDE
:101F00004CFED8FF7103AB01CFFA7DFBE505180845
:101F100040FBDDF4D301550CD301DDF440FB180880
:101F2000E5057DFBCFFAAB017103D8FF4CFEBEFF88
:101F3000A3003A00BFFF0000000000000100010004
:101F40000600000200010000040000001000000074
:101F5000100000000000E02E7017B80BE80300002E
:101F6000000000000200000010000000000000005F
:101F7000030000000000000000000000000000005E
:101F8000000000000000060000000000010000004A
:101F9000B01F0008000000205800000028010008C1
:101FA00008200008580000207006000044010008C6
:101FB00002040608000000000102030401020304F9
:101FC0000607080900080140001001400010014008
:101FD0000000000000000000000000000438014084
:101FE00000000000100000000000000000000000E1
:101FF0008000000000000000000000000000000061
:082000000020000000000000B8
:04000005080000ED02
:00000001FF
